:0800000013C0FECF4AC0FCCF83
:10000800FBCFFACFF9CFF8CFF7CFF6CF000000003B
:1000180000000000000000000C00030014000000B5
:10002800F894EE27ECBBE5BFF8E1A4B7A77FA4BF1F
:10003800F1BDE1BD8DE0A2E0ED938A95E9F780E49A
:10004800A0E6ED938A95E9F7E0E2F0E0C8953196ED
:10005800802DC8953196902D0097B9F0C8953196A6
:10006800A02DC8953196B02DC8953196102CC895FD
:1000780031966E2F7F2FF02DE12DC89531960D9278
:100088000197D9F7E62FF72FE1CFEFE9EDBFC0E7EA
:1000980022C0EA93FA93EFB7EA93E0E0B099E1E07F
:1000A800BE2ECC24E0E0B199E1E0DE2EEE24B29B36
:1000B80006C0E0E0E0937000E093710005C000D155
:1000C800E0937000F093710033244424E991EFBF6A
:1000D800F991E9911895E0E8E6BDE1E0E6BDE8E0D0
:1000E800E8BBE0E3E7BBE0E0EFBDE3BFE2BFE6BFAC
:1000F800E9BDE0E2EBBFE0E0E5BFEFE0E5BBE0E251
:10010800EABFE0E0E9BFE0E8E8B9E0E0E3B9789405
:10011800DAD029F4DCD019F4DED01097A1F0D3D0CE
:1001280021F4D5D011F4DCD071F0CDD029F4DBD096
:1001380019F4D1D0109739F0C6D021F4D4D011F4E5
:10014800CFD009F002C0AA249924D1D029F4BFD075
:1001580019F4C1D0109709F023C0E1E09E1618F0F9
:10016800E3E09E1608F00DC0E0EAFFE0E315F405B1
:1001780024F0A6D03E0E4F1E02C0EAE0AE2EE2E00A
:100188009E2EE3E0E91541F4EBE0AE2EB4D0E51580
:10019800F60511F4E1E09E2EE1E0E91508F0AED095
:1001A800A6D021F494D011F49BD009F009C0E2E064
:1001B8009E1628F0EAE0AE2EE3E09E2E01C09ED007
:1001C80096D029F490D019F486D0109709F003C07E
:1001D80095D0E1E09E2E8BD021F485D011F480D00B
:1001E80009F008C0E3E0E91511F4AA2403C086D099
:1001F800E1E09E2EE1E0EA15A1F47DD05E166F06DF
:100208007CF4E4E1F0E07DD082D01CF086D089D087
:10021800FBCF8ED091D01CF080D083D0FBCF01C013
:100228008ED0EBE0EA1599F466D05E166F0674F48A
:1002380047D067D06CD01CF070D073D0FBCF78D08B
:100248007BD01CF06AD06DD0FBCF01C078D0AA203B
:10025800C9F4002405140604A4F4E52DF62D7497BA
:100268005E2E6F2E65D068D01CF057D05AD0FBCFC9
:10027800C498772488244BD01CF04FD052D0FBCFA1
:1002880001C05DD0EAE0EA15C9F4002405140604AB
:10029800A4F4E52DF62D31975E2E6F2E49D04CD063
:1002A8001CF03BD03ED0FBCFC498772488242FD0B5
:1002B8001CF033D036D0FBCF01C041D029CFFFCFBF
:1002C800E1E0F0E0089500240B140C0408950024E4
:1002D8000D140E040895A0917000B0917100089556
:1002E800FADF11970895ECDFED15FE050895E8DFB4
:1002F800EB15FC050895E0E1F7E20895E1E0AE2E84
:1003080008955E0E6F1EC498772488240895F3DF3D
:10031800E519F609E715F805089581E08A95F1F7DA
:100328000895E72DF82DEC59FF4F7E2E8F2E089556
:10033800C49A772488240895571468040895E4E635
:10034800F0E0FA93EA9300C0E991F991309639F018
:1003580084EF91E00197F1F7A8953197C9F70895CF
:00000001FF
